:020000040000fa
:10000000f81f00204d2d00007b2f00006b330000f7
:1000100000000000000000000000000000000000e0
:100020000000000000000000000000001724000095
:10003000000000000000000017240000bd38000090
:100040001724000017240000593500001724000071
:10005000cd360000172400001724000017240000ec
:1000600017240000172400001724000017240000a4
:100070001724000017240000172400001724000094
:100080001724000017240000172400001724000084
:1000900017240000172400000d1500000d150000a6
:1000a0000d1500000d150000a5160000a516000096
:1000b000a5160000a5160000172400001724000054
:1000c00017240000172400005534000017240000f6
:1000d0001724000017240000172400001724000034
:1000e0001724000017240000172400001724000024
:0400f00017240000d1
:020000040000fa
:1000f400401801000200030084468ef30088744710
:10010400f8b5c046f8bc08bc9e467047a12f000055
:10011400f8b5c046f8bc08bc9e4670477d2f000069
:020000040000fa
:08012400bc1000000100000006
:020000040000fa
:10012c004d6f64756c6520736179733a202573008b
:10013c002b455252000000004461746120776572b7
:10014c0065206e6f74206265656e20706f737465c8
:10015c0064202d3e20627574746f6e5f73746174cd
:10016c0065203d2025640d0a0000000041542b55ec
:10017c00545820350d000000000000000000000065
:10018c000000000000000000000000000d0a4461a7
:10019c00746120706f7374656420746f206d6f646c
:1001ac00756c653a2025730d0a000000205f5f5fb7
:1001bc005f5f205f5f5f5f5f205f5f5f5f5f205f00
:1001cc005f5f5f5f20202020202020202020205fe8
:1001dc00205f205f205f5f5f5f5f205f5f5f205f5e
:1001ec005f5f202020202020202020202020205f46
:1001fc005f5f5f5f205f5f5f5f5f205f5f5f5f5f81
:10020c00205f5f5f5f5f200d000000007c202020de
:10021c005f5f7c20205f20207c2020205f5f7c2083
:10022c0020205f5f7c2020205f5f5f2020207c20cf
:10023c007c207c207c2020205f5f7c2020207c5f29
:10024c0020207c20202020205f5f5f2020207c5fee
:10025c002020205f7c2020205f5f7c20202020201d
:10026c007c20205f20207c0d000000007c5f5f2044
:10027c0020207c2020205f5f7c5f5f2020207c2062
:10028c0020205f5f7c20207c5f5f5f7c20207c20b7
:10029c007c207c207c5f5f2020207c207c207c5f6d
:1002ac007c207c5f2020207c5f5f5f7c20202020d6
:1002bc007c207c207c2020205f5f7c207c207c208c
:1002cc007c2020205f5f7c0d000000007c5f5f5f66
:1002dc005f5f7c5f5f7c20207c5f5f5f5f5f7c5f2c
:1002ec005f5f5f5f7c2020202020202020207c5f0f
:1002fc005f5f5f5f7c5f5f5f5f5f7c5f5f5f7c5fab
:10030c005f5f5f5f7c202020202020202020202089
:10031c007c5f7c207c5f5f5f5f5f7c5f7c5f7c5f72
:10032c007c5f5f7c2020200d000000000d00000091
:10033c00205f5f5f5f5f2020202020202020202076
:10034c002020202020202020202020202020205f62
:10035c00202020205f202020202020202020205f13
:10036c005f5f5f5f205f5f5f5f2020202020205f4a
:10037c00202020202020200d000000007c20205f69
:10038c0020207c5f5f5f205f205f205f205f5f5fce
:10039c00205f5f5f205f5f5f205f7c207c20207c84
:1003ac00207c5f205f205f2020207c5f2020205f4e
:1003bc007c202020205c205f5f5f7c207c5f205fa6
:1003cc005f5f200d000000007c2020205f5f7c2000
:1003dc002e207c207c207c207c202d5f7c20205fac
:1003ec007c202d5f7c202e207c20207c202e207ccd
:1003fc00207c207c202020207c207c207c20207cc9
:10040c0020207c202e277c20205f7c202e277c0d1a
:10041c00000000007c5f5f7c20207c5f5f5f7c5f66
:10042c005f5f5f5f7c5f5f5f7c5f7c207c5f5f5f9b
:10043c007c5f5f5f7c20207c5f5f5f7c5f20207c2b
:10044c00202020207c5f7c207c5f5f5f5f2f7c5fa7
:10045c005f2c7c5f7c207c5f5f2c7c0d000000009f
:10046c002020202020202020202020202020202080
:10047c002020202020202020202020202020202070
:10048c00202020202020207c5f5f5f7c20202020eb
:10049c002020202020202020202020202020202050
:1004ac00202020202020200d000000002d3e204c7c
:1004bc004153542046572055504441544520253033
:1004cc0032642e253032642e2025303464202530c1
:1004dc0032643a253032643a253032640d0a000019
:1004ec002d3e20496e697469616c697a6174696f1b
:1004fc006e2c206f6e65206d6f6d656e7420706c48
:10050c0065617365203a2d290d0a0d00436f6d6de1
:10051c00616e6420706f7374656420746f206d6fee
:10052c0064756c653a2025730a0000002d3e204945
:10053c006e697469616c697a6174696f6e204f4b76
:10054c000d0000000d0a2d3e2053797374656d204b
:10055c0074696d6520253032642e253032642e206e
:10056c002530346420253032643a253032643a2503
:10057c003032640d0a0000000d0a54656d7065720e
:10058c0061747572653a20253032642e25303264e0
:10059c000d0a48756d69646974793a2025303264a6
:1005ac002e253032640d0a427574746f6e2073748c
:1005bc006174653a2025640d0a0000002d3e204729
:1005cc006f696e6720746f20736c656570203a2daf
:1005dc00280d00000d0a2d3e20426f6172642069c7
:1005ec0073206177616b656e6564203a2d290d006f
:1005fc0041542b4d4f44453d300d000041542b5080
:10060c004f52543d320d000041542b44464f524d35
:10061c0041543d310d00000041542b445554594375
:10062c0059434c453d300d0041542b4445564144f3
:10063c0044523d30393339376333330d00000000f9
:10064c0041542b4445564555493d323430333233b1
:10065c00323733636133356336610d0041542b41be
:10066c005050534b45593d346630396532643937f7
:10067c003634313230313539613764666438343070
:10068c00613163343733360d0000000041542b4e7a
:10069c00574b534b45593d6565313139333863619f
:1006ac00616162396261323064353831646364335c
:1006bc00383032626638310d0000000041542b4155
:0806cc0044523d310d00c0460f
:020000040000fa
:1006d400f0b59bb00390029115001c0020b1836912
:1006e40004930bb902f0fcf8964b029a9a4260d13b
:1006f400039b5b680293029b9b891b0767d5029b44
:100704001b690493002b62d000220d92202208abb7
:100714005a76302204959a76049d2b78002b60d16a
:10072400049bee1a66b13300049a0299039802f00e
:1007340077fb431c00d15be10d9b9e1904930d963e
:100744002b78002b00d153e1012208ae5242726093
:100754005322002304a97c4f521801350893f360f7
:10076400b3601370223705222978380003f048f962
:100774006a1c002839d13068c30604d553232021cc
:1007840004afdb191970030704d553232b2104afdd
:10079400db1919702b782a2b2fd000200a21f3683b
:1007a4002a78303a092a00d870e000282cd0f36067
:1007b4002ae0664b029a9a4202d1039b9b6899e70e
:1007c400634b029a9a4296d1039bdb6892e70299a3
:1007d400039801f0cbfb002896d0012040421bb0c7
:1007e400f0bd252b9cd0013597e70123c01b834026
:1007f400316815000b433360b5e72368211d002bd6
:100804003edbf36015000c002b782e2b0ad16b789d
:100814006a1c2a2b42d122680235231d002a3adba6
:100824001c007260484f297828370322380003f0ef
:10083400e7f830b14023c01b8340326801351343cd
:100844003360414f6b1c38002978532506222c3025
:100854000493317603f0d4f8327e04abed18692aa0
:1008640032d03ed8582a00d1c9e029d8002a00d174
:10087400f2e0522504abed1801232a700c9350e0ea
:100884005b42f360022303433360bbe74b43013510
:100894009b18012084e701225242c1e7002315007e
:1008a4000a201a00736029783039092903d9002bea
:1008b400b8d07260b6e74243013552180123f2e71b
:1008c400632a26d0642ad4d10899221d0b062ed57a
:1008d40023681400002b02da2d225b422a700a22bc
:1008e40045e0732a00d1b9e008d86f2a24d0702ad1
:1008f400bfd1202332681343336003e0752a1bd031
:10090400782ab6d15523782204a95b181a701137b6
:1009140079e0522504abed18237804342b700123bd
:1009240033615323002204a95b181a7042e0236840
:100934004906ced51bb2cce7089b211d180609d564
:1009440023680be06c370000043300008c37000090
:100954004c3700005b06f3d523689bb20c006f2a6a
:1009640069d00a225321002004ad4919087009995d
:100974000a91002900da97e00420089d8543089530
:10098400002b5ad1002900d090e0532504abed1878
:10099400082a0ad1089b0593db0706d5099a0c9b04
:1009a4009a4202dc3023013d2b70532304aa9b1886
:1009b4005b1b0c93404b07aa009308a9029b039866
:1009c40001f046fb431c13d00c9b2a0002990398a8
:1009d40002f026fa431c0bd0089b002505939b07c5
:1009e40056d4079a0b9b934200da13005a1c56d133
:1009f400029b0d989b895b0600d4f0e6ede6552337
:100a040004a95b181a70089a211d130601d52368de
:100a140003e05306fbd523689bb20c00d10702d533
:100a240020210a4308921022002b9bd120210898f0
:100a34008843089096e7082294e7532504a96d1883
:100a4400b3fbf2f1100048431b1afb5c013d2b7011
:100a54000b000029f4d19be73261abe7256872688b
:100a640000212800271d02f0cbff08b1401b706055
:100a7400099b3c0005930c9353e7292204a9012305
:100a840052180398029902f0cbf9431cb0d00135f7
:100a94000b9b079a05939b1a9d42eedba1e70d9ae7
:100aa400d31805920d9337e6002bc6d1522504ab1b
:0c0ab400ed183b782b706be7252e00003e
:020000040000fa
:100ac000d80300201c00000000000000e402002009
:100ad00030000000010000004c28000050280000f9
:100ae00054280000582800005c28000060280000fe
:100af00064280000682800006c28000070280000ae
:100b00007428000078280000f40300200c00000086
:100b1000010000004d61792020392032303231004f
:100b20000c040020090000000100000031303a34bc
:100b3000383a323300000000980300202000000003
:100b40000000000000000020600000000000000025
:100b5000000400200c0000000000000044030020fe
:100b60002c000000000000001403002030000000f2
:100b700000000000600000200c00000000000000e9
:100b800018040020080000000000000030040020cd
:100b90000300000000000000b80300202000000057
:100ba000000000001504002001000000000000000b
:100bb00016040020010000000000000017040020bf
:100bc00001000000000000003304002001000000cc
:100bd00000000000340400200100000000000000bc
:100be000a4020020400000000000000035040020a6
:100bf0000100000000000000360400200100000099
:100c00000000000037040020010000000000000088
:100c1000700300202800000001000000fc05000017
:100c20000806000014060000240600003406000038
:100c30004c0600006806000098060000c806000088
:100c4000000000006c0000206800000000000000b0
:100c500020040020040000000100000044020020e5
:100c600044020020600000000100000000000000bd
:100c70006c3700008c3700004c370000000000008b
:100c80000000000000000000000000000000000064
:100c90000000000000000000000000000000000054
:100ca0000000000000000000000000000000000044
:100cb0000000000000000000000000000000000034
:100cc00000000000000000000000000024040020dc
:100cd00004000000000000002804002004000000c0
:100ce00000000000d80000206c010000010000009e
:100cf00043000000000000000000000000000000b1
:100d000000000000000000000000000000000000e3
:100d10004300000000000000000000000000000090
:100d200000000000000000000000000000000000c3
:100d30004300000000000000000000000000000070
:100d400000000000000000000000000000000000a3
:100d50004300000000000000000000000000000050
:100d60000000000000000000000000000000000083
:100d70004300000000000000000000000000000030
:100d80000000000000000000000000000000000063
:100d90004300000000000000000000000000000010
:100da0000000000000000000000000000000000043
:100db00043000000000000000000000000000000f0
:100dc0000000000000000000000000000000000023
:100dd000ed3900000d380000000000007c1c000010
:100de000293b0000283b0000283b0000283b000076
:100df000283b0000283b0000283b0000283b000067
:100e0000283b0000283b0000ffffffffffffffff24
:100e1000ffffffffffff000001004153434949006e
:100e200000000000000000000000000000000000c2
:100e30000000000000000000000041534349490049
:100e400000000000000000000000000000000000a2
:100e5000000000000000000000000000d40000209e
:100e600004000000000000002c040020040000002a
:100e700000000000000000000000000022222222ea
:020000040000fa
:100e8000f0b5ce4600b58eb0e1235b020a93002494
:100e90000c9402260b960d94b34d29000aa800f07d
:100ea00055fd0021b14802f029fe44f600330693b7
:100eb000089407960994290006a800f0b3fc0022c4
:100ec000ab49012002f034fbaa4b0093aa4bab4a7a
:100ed0007021ab4802f0f7fdaa4e300000f048fe4a
:100ee000a94d2900300002f01ffda84c2100a848a0
:100ef00002f0f8fd280002f021f9ab68a3602b682e
:100f0000053323606b6863602b6923616b696361e0
:100f1000eb68e360ab69a3610621200001f026fec7
:100f20009c4c20000c3002f08dfd20006c3002f053
:100f300089fd99484c3002f085fd98482c3002f02c
:100f400081fd974c25000c35280002f07bfd200028
:100f5000103002f077fd20005c3002f073fd914c00
:100f60002000283002f06efd2000743002f06afd8f
:100f70008d48403002f066fd280002f063fd280035
:100f800002f060fdf38840f26c7c634432790132f8
:100f9000f178864c20000c303578029575780195f3
:100fa000b578009502f0b2fb2000403002f04afd17
:100fb0007f4c804e804b343304937f4b1c3305931e
:100fc00036e07e4b1b789b007d4a9958b1b177483b
:100fd0006c3002f09bfb794d2b789b00784a9f5830
:100fe000380002f077fd0100380001f0ddfc2b78bd
:100ff00001332b70c82002f01bfd19e000226f4b5b
:101000001a7001216f4802f019f865480c3002f09f
:1010100019fd40f2f41002f00bfd0122644b1a702e
:1010200006e069480c3002f00dfd0222604b1a7098
:101030002378052bfdd89b00f3589f46634b1a7805
:10104000634b1b781343002bf2d0604b1b78002bb3
:1010500043d14d4f380001f0b1ff7b6940f26c7c09
:1010600063443a690132f9685748814624303d6843
:1010700002957d680195bd68009502f047fb404fe1
:10108000380001f07bf9534d2b789c46bb7c7a7c71
:10109000397c2d3948465830814660460190ff7ca6
:1010a0000097484602f032fb2b789bb34a4b1878e6
:1010b00001231843484b1870484901f037fa64205f
:1010c00002f0b6fc01f0ecfa0322394b1a7000234f
:1010d0003f4a13703d4a1370aae72c4f380001f0c5
:1010e0006dff3b683b2b05dd284a3b3b1360536893
:1010f00001335360254b5b685a1d3b2a07dd363ba5
:10110000224a53600221214801f030fda1e71f4b24
:101110005a60f7e7304b187801239843cae70598df
:1011200002f090fc02f0bcfb02f0acfb02f09cfb76
:1011300002f08cfb04221e4b1a7079e702f002fccd
:1011400005221b4b1a7073e702f02cfc02f01efc08
:1011500002f010fc02f002fc049802f073fc012281
:10116000134b1a7064e7c04640420f0081350000ff
:10117000b12e0000ed360000152b0000313a0000c2
:10118000c0000020b40000206c000020900000206f
:10119000893a0000ac0100002c020000ac02000003
:1011a0002c030000ac0300002c040000ac04000081
:1011b00034040020bc390000ac05000033040020da
:1011c00070030020360400202c05000015040020c8
:1011d000160400201704002037040020d00000204f
:020000040000fa
:1011e000f0b51f0085b005000c00160000920197b5
:1011f00002900391002f00d0d5e08e424ed93000ee
:1012000001f0d8ff58b120232a001b1ada4084408d
:101210001300864085402343009603930295009b6c
:1012200003991a0cb1fbf2f615006b4637007543b3
:101230001b884d1b5f4302992d040c0c2543310084
:10124000af4208d9009c01392d19ac4203d8af42f6
:1012500001d9b11e2d19ef1bb7fbf2f46243bf1a7f
:101260006a46634312893f043a432600934208d9f1
:10127000009d013e5219954203d8934201d9a61e02
:1012800052190904d31a31430a9a1ab1c3401360a0
:10129000002353600800019905b0f0bd1eb9012379
:1012a000b3fbf6f30093009801f084ffc0bb009bf2
:1012b000e41a01230193009b1a0cb4fbf2f116000f
:1012c0006b460d004e431b88a41b5d43029e240405
:1012d000360c34430f00a54208d9009e013fa419e3
:1012e000a64203d8a54201d98f1ea419641bb4fbe2
:1012f000f2f67243a41a6a46734312892404144313
:101300003100a34208d9009a0139a418a24203d897
:10131000a34201d9b11ea4183f04e31a3943b3e72d
:10132000009b20228340009323002f00121ad340f9
:101330008540d740009a0295110cb3fbf1f56a463f
:101340002e0012888440944656430a006a4327437d
:101350009b1a1b043a0c13432a009e4208d9009c96
:10136000013a1b199c4203d89e4201d9aa1e1b199f
:101370009e1bb6fbf1f5644669436c43761a36044e
:10138000bfb237432b00bc4208d90099013b7f18fc
:10139000b94203d8bc4201d9ab1e7f1812041a43cc
:1013a0003c1b019287e78f4209d90a9b002b00d191
:1013b000a9e0186059600023019319006ae738001a
:1013c00001f0f8fec8b9a74202d30100ae4208d826
:1013d000ae1bb542ad410121e41b6d42631b03937b
:1013e00002960a9b0193002b00d153e7029a1a60e0
:1013f000039a5a60002301934ce720231b1a0093a1
:101400003b003700009a8340d7401f432300d3405e
:101410002a0000998440ca40224394463a0cb3fb08
:10142000f2f41100864085406143019626005b1a64
:1014300061460295bdb26e43090c1b040b432100ab
:101440009e4207d9db1901399f4203d89e4201d938
:10145000a11edb199e1bb6fbf2f462436346b61a6b
:101460006a46654393819289360416432300b54248
:1014700007d9f619013bb74203d8b54201d9a31edb
:10148000f619090419436b469c88019b721b94460c
:101490001a0c23008eb20d0c6c43734355437243f8
:1014a0001e0c1219b218944202d9802464022d191c
:1014b000140c9bb212046519d218ac4503d30bd19e
:1014c000029b934208d2019bed1bd61ab242924175
:1014d0005242ad1a320001390a9b0193002b00d110
:1014e000d8e6029b009c9a1a63465d1b029b9342be
:1014f000bf417f42ed1b2b00c240a340c5401a43b1
:0a1500000a9b24c376e70a9b56e716
:020000040000fa
:02150a00704728
:020000040000fa
:10150c0010b5634b9b7dbbb1614b5b8b9b0714d5bb
:10151c00604bff212022995402212122995420232f
:10152c005c4ad35c5bb2013300d181e02023594a81
:10153c00d35c062b00d193e010bd554b5b8bdb07c6
:10154c0007d5544bff212022995402212122995472
:10155c00e5e74f4b5b8b5b0707d54e4bff212022fa
:10156c009954012121229954d9e72023494ad35c6b
:10157c005bb2032b3ed0042b0ed0022bcfd11369c0
:10158c0023b19088002101f015fbc8e7414b9888e6
:10159c00012101f00ffbc2e73e4a936912699342a5
:1015ac0008d03c4a9168581c9061c95c2823384a81
:1015bc00d154b4e7374b5b6973b1364b9b885b00f6
:1015cc0001221343324a5362d369002bfcd103210d
:1015dc002023304ad154a2e72d4a5168c0239b02e4
:1015ec000b435360d369002bfcd106212023294add
:1015fc00d15494e7274a5369013bd2699a4209d0e6
:10160c00244bd968da69501cd86128232048c35c64
:10161c008b5484e71e4a5168e023db020b43536072
:10162c00d369002bfcd1062120231a4ad154e7e7b9
:10163c0000212023d154164a5168c0239b020b432e
:10164c005360d369002bfcd18322114b1a76114bba
:10165c005b6a002b00d16fe70e4a906a98476be7e4
:10166c001300002220215a5421215a548322084b62
:10167c001a76190030224b8b1340102bfbd1054be3
:10168c005b6a002b00d157e7024a906a984753e7f0
:08169c00000400424403002099
:020000040000fa
:1016a400f8b5ce46474680b55b4b9b7dbbb15a49e6
:1016b4000a7ed2b28b7d5bb2002b14db564a137eba
:1016c400dbb2927dd20701d5db075dd4524a137e8b
:1016d400dbb2927d520702d55b0700d56ce00cbcef
:1016e40090469946f8bd52b2002ae7da4a4b5b8b22
:1016f40007221340002be1d0484ce38501f092fe11
:101704008422454b1a7500222c23e254636a002b71
:10171400d4d0424a906a9847d0e78368591c8160c4
:101724006146cb5c1385b168137e2b4211d08c4289
:101734000fd953683b40012befd143469b68994630
:10174400591c434699604b465b0061465b5a1385be
:10175400e9e7324b9a685b689a42b7d32f4b002271
:101764001a755a6001212c4a1175db68002badd023
:101774002a4a10699847a9e7284a9069136a5c1ca9
:1017840014625b00195231e0244b1b7d002b9dd069
:10179400224b9a685c68204b1b7edb07d9d5a2429a
:1017a400d7d21e4b1b689c461b4a07271b4b9846e7
:1017b40018001e000125bce72c23184ad35c002b1b
:1017c40000d18ce7154b1a6adb699a4200d386e78d
:1017d400114b198d89b25a6807231340012bcbd0c2
:1017e4000e4b98691a6a541c1c6281540b4b1a6a7a
:1017f400db699a4200d072e7084b00222c215a542c
:10180400da618421044a11755b6a002b00d166e712
:10181400024a906a984762e70008004214030020d5
:020000040000fa
:1018240070b506000d00434b1c7de4b22c229b5c7a
:10183400dbb2002b79d1002c00d079e0002875d0e0
:101844000068002872d001b93b4d03019d423bd38f
:10185400010b00052a00002301f02efc80235b020b
:10186400181a0021002861d0344a13680224a343c3
:101874001360d369002bfcd180b2304b988173681c
:10188400022b42d02d4a136849032d481840802367
:101894005b040343194311605168b368f068034360
:1018a400284801400b4371680b435360234ad369b2
:1018b400002bfcd1214a136802210b431360d36926
:1018c400002bfcd1012431e0c3009d420ad3410b1b
:1018d400c0042a00002301f0effb80235b02181ae6
:1018e4000221bfe743001b189d421fd3c02292026e
:1018f4000023002101f01efb2a00002301f0dcfb81
:1019040080235b02181a0421ace70c4a13684903cc
:101914000b480340194311605168b368f0680343ee
:10192400472081430b435360c0e70024200070bd6f
:101934001c00fbe71403002040420f000008004293
:08194400ff1ffff0b8dffffff9
:020000040000fa
:10194c0070b505000e00002800d176e00468002078
:10195c00fcb301b93b4e23019e423bd3210b200526
:10196c003200002301f0a4fb80235b02181a002133
:10197c00002864d0344a13680224a3431360d3694b
:10198c00002bfcd180b2304b98816b68022b44d079
:10199c002d4a136849032d48184080235b040343e8
:1019ac00194311605168ab68e8680343284801404b
:1019bc000b4369680b435360234ad369002bfcd15a
:1019cc00214a136802210b431360d369002bfcd10d
:1019dc00012070bde3009e420ad3610be00432008b
:1019ec00002301f065fb80235b02181a0221bfe77c
:1019fc0063001b1900209e42ebd3c02292020023ed
:101a0c002000002101f092fa3200002301f050fb7b
:101a1c0080235b02181a0421aae70b4a13684903b6
:101a2c000a480340194311605168ab68e8680343e6
:101a3c00472081430b435360bee70020c9e70020d9
:101a4c00c7e7c04640420f00000c0042ff1ffff0ea
:041a5c00b8dffffff1
:020000040000fa
:101a6000f7b58a8905000c0013075ed44b68002b7c
:101a700004dc0b6c002b01dc0020febde76a002fac
:101a8000fad000232e682b6041f200031a4092b373
:101a9000606da3895b0705d56368c01a636b0bb1e2
:101aa000236cc01a0200216a00232800e76ab847a5
:101ab000a189431c06d12b681d2b30d82b4ada4054
:101ac000d3072cd50023636023692360cb0404d59e
:101ad000431c01d12b6803b96065616b2e6000293e
:101ae000cad023004433994202d0280000f094fc6d
:101af00000206063c1e70123216a2800b847431c26
:101b0000c7d12b68002bc4d01d2b01d0162b01d1bf
:101b10002e60b1e74023a2891343a381ade74023a0
:101b20000b430120a3814042a7e70f69002fa3d0f8
:101b30000b680f60db1b01930023920700d14b69f8
:101b4000a360019b002b00dc96e7019b3a00216a11
:101b50002800a66ab047002803dc4023a28913436b
:101b6000dfe7019b3f181b1a0193eae701004020c1
:020000040000fa
:101b7000f8b507003d4b1b78202b34d0303b9a0042
:101b80009b185b00dbb239494a78303a9b18bb702e
:101b9000cb78202b29d0303b9a009b185b00dbb21e
:101ba00032490a79303a9b187b708b79202b1ed0f2
:101bb000303b9a009b185b00dbb22c4ad279303a5a
:101bc0009b183b702a4b1b78202b08d028494b1cb4
:101bd0000c311a78202a02d001338b42f9d1254ddd
:101be0000024234e0ae00023cde70023d8e700239a
:101bf000e3e70134e4b204350c2c08d003223100b1
:101c0000286801f093fd0028f3d13c71f1e7184bef
:101c10001b79202b28d0303b98001b185b00d8b2d2
:101c200013494b79303bc018c0b2f870ca79303aca
:101c300040f2e8335a430b7a303b64246343d318b1
:101c40008a7ad2184b7a303b99005b185b00d21825
:101c500092b2094bd318fb80303a92b2397901f035
:101c60002bf838720120f8bd0020d9e70c040020c1
:0c1c7000f4030020e402002064f8fffff1
:020000040000fa
:101c7c000020202020202020202028282828282050
:101c8c002020202020202020202020202020202048
:101c9c0020881010101010101010101010101010b0
:101cac0010040404040404040404041010101010a0
:101cbc00101041414141414101010101010101016a
:101ccc0001010101010101010101010110101010bc
:101cdc00101042424242424202020202020202023c
:101cec000202020202020202020202021010101090
:101cfc0020000000000000000000000000000000b8
:101d0c0000000000000000000000000000000000c7
:101d1c0000000000000000000000000000000000b7
:101d2c0000000000000000000000000000000000a7
:101d3c000000000000000000000000000000000097
:101d4c000000000000000000000000000000000087
:101d5c000000000000000000000000000000000077
:101d6c000000000000000000000000000000000067
:011d7c000066
:020000040000fa
:101d8000f0b5d6464f464646c0b5bff35f8f62b644
:101d9000374b40f200301a58364d2a40c021090412
:101da0000a431a5040f2040a52461a6040f20436be
:101db0009a59ff208243c0273a439a5110221a6051
:101dc00010369a592a400a439a518022d2031a6047
:101dd0009a591202120ac0242406a14622439a519b
:101de000802212041a6040f218329e5886433e4305
:101df0009e50802676041e609e581f4ca0462640aa
:101e00004cf2000c644626439e508026b6041e60a9
:101e10009e582e400e439e508026f6041e609e580b
:101e20003602360a4c4626439e50802212051a601e
:101e300040f21c369a598243100038439851802250
:101e400052051a609a5940460240604602439a5130
:101e5000802292051a6040f220301a58154029431a
:101e6000195052465a601cbc90469946a246f0bd95
:0c1e700000e100e0ffff00ffff00ffffab
:020000040000fa
:101e7c000222374b1a760022364b1a74364a374bed
:101e8c005a62190008224b681a42fcd14121802366
:101e9c00324ad15010008021402243581a42fcd0c3
:101eac002b4b20225a633f221a6318003c21042238
:101ebc00435c1342fcd102212c23254ad15410003f
:101ecc003c210222435c1342fcd1214840210322d5
:101edc00435c1340032bfbd1214a204b1a6219009f
:101eec0004224b681a42fcd140218c231b4ad1504e
:101efc0010008c21402243581a42fcd04021ac23c4
:101f0c00164ad1501000ac21402243581a42fcd042
:101f1c004021b023114ad1501000b0214022435827
:101f2c001a42fcd04021b4230c4ad1501000b421e9
:101f3c00402243581a42fcd04021b823074ad150c2
:101f4c001000b821402243581a42fcd07047c046ba
:101f5c00001000400014004005010400001c00406b
:041f6c000701400029
:020000040000fa
:101f7000344b70b51d6806000c0025b1ab6913b970
:101f8000280000f0affc304b9c420fd16c680c2352
:101f9000e25e93b219072cd4d90611d40923336019
:101fa000402301201343a381404270bd274b9c4234
:101fb00001d1ac68ebe7264b9c42e8d1ec68e6e740
:101fc0005b0712d5616b41b123004433994202d0c3
:101fd000300000f021fa002363632422a389934395
:101fe000a38100236360236923600823a28913432c
:101ff000a38123695bb940f2802140f20022a389ca
:102000000b40934203d02100300000f0c1fb0123bc
:10201000a28913408bb10023a36063695b42a36173
:1020200023690020002bc0d10c23e25e1306bcd52f
:1020300040231343a3810138b7e7920700d46369b3
:10204000a360ede7200400206c3700008c3700000f
:042050004c37000009
:020000040000fa
:10205400f7b5150001938a680b6900900c00934250
:1020640000da130022002b60433212780ab10133e4
:102074002b6023689b0602d52b6802332b6006274e
:1020840023681f403fb3230043331b785a1e9341f8
:102094002268920630d42200019943320098089ea7
:1020a400b047431c25d0062320682a68e168034012
:1020b4000025042b03d18d1aeb43db171d40a368c5
:1020c4002269934201dd9b1aed180027bd4220d1fd
:1020d400002010e00137e3682a689b1a9f42d2da95
:1020e40022000123193201990098089eb047431c2d
:1020f400f0d101204042febd3020e1184331087088
:1021040021005a1c45310978a21843320233117058
:10211400c1e7220001231a3201990098089eb047b2
:08212400431ce6d00137d1e7ae
:020000040000fa
:10212c0070b505000e0018b183690bb900f0d4fb33
:10213c00ab69ac6813b9280000f0cefb294b9c426c
:10214c0019d16c680c23e25e42f200031a4205d1ed
:10215c001343a381226e244b13402366a3891b07d0
:10216c0001d52369fbb921002800fff7fbfed0b194
:10217c000120404270bd1d4b9c4201d1ac68e1e78f
:10218c001b4b9c42ded1ec68dce7013b0136a360c3
:10219c00002b04daa269934216db0a2914d02368b7
:1021ac005a1c226019703178a3680029edd1013bcb
:1021bc00a360002b0fda22000a21280000f01af885
:1021cc00431cd5d00a20d5e72200280000f012f8d5
:1021dc00431ce8d1cce70a2023685a1c22601870f3
:1021ec00c8e7c0466c370000ffdfffff8c370000ec
:0421fc004c3700005c
:020000040000fa
:10220000f8b505000e00140018b183690bb900f091
:1022100069fb274b9c4230d16c68a369a360a389fa
:102220001b0734d5236993b30c23e25e42f200030b
:10223000f7b2f6b21a4234d023682269981a636959
:10224000984204db2100280000f0e4fc28bba368ce
:102250000130013ba36023685a1c22601f70636930
:10226000984204d0a389db0719d50a2e17d1210083
:10227000280000f0cffc90b10fe00e4b9c4201d142
:10228000ac68cae70c4b9c42c7d1ec68c5e721009b
:102290002800fff76dfe0028c6d0012676423000e8
:1022a000f8bd1343a381226e044b13402366c3e79a
:1022b0006c3700008c3700004c370000ffdfffff59
:020000040000fa
:1022c000032370b5cd1c9d43083506000c2d1cd290
:1022d0000c25a9421bd8300001f0b7fa254a146832
:1022e0002100c1b9244c23681bb9300001f05efa0b
:1022f00020602900300001f059fa431c2dd10c2335
:102300003000336001f01dfb03e0002de1da0c2307
:102310003360002070bd0b685b1b1bd40b2b03d9f3
:102320000b60cc18256003e08c420fd1636813600a
:10233000300001f006fb200007220b30231d9043e4
:10234000c31a002be6d05a42e250e3e74b686360c1
:102350000c00ede70c004968c3e70323c41c9c4351
:10236000a042dfd0211a300001f020fa431cd9d15d
:0c237000c5e7c04624040020280400201b
:020000040000fa
:10237c00f0b585b0040002ae00230293b38001ad2a
:10238c0035232b7017236b70290001f08ffb012074
:10239c00e36898475c232b7024236b702900200082
:1023ac0001f084fb0d20e3689847062231002000e1
:1023bc0063689847327812027378134342f21072b2
:1023cc005a4312146421b2fbf1f0c0b2a07464271a
:1023dc007843121ae274f3781b0232791a4344f2ee
:1023ec005c4353431b14b3fbf1f1cab222747a431e
:1023fc009b1a6374b0232b7098236b7029002000f8
:0a240c0001f054fb012005b0f0bd03
:020000040000fa
:02241600fee7df
:020000040000fa
:1024180070b5050079b10c1f2368002b00dae418a9
:10242800280001f00efa1c4a13682bb96360146087
:10243800280001f082fa70bda34209d9216860180a
:102448008342f3d118685b6841182160eee71300f6
:102458005a680ab1a242fad919685818a0420bd191
:1024680020680918581819608242e1d1106852682a
:10247800411819605a60dbe7a04202d90c232b608f
:10248800d6e721686018824203d110685268411863
:0c249800216062605c60cbe7240400203f
:020000040000fa
:1024a4001e4a1f4b70b50021934203d219700133a9
:1024b4009342fbd1002503261a4803684168b3b947
:1024c40059b383680c30bbb100230022845c9c5454
:1024d40001328a42fad333000b405a1e93418908d1
:1024e40059188900401803684168002be8d08268b5
:1024f4000c303ab90029e0d059181d7001338b42d1
:10250400fbd1dae70029e0d133000b405a1e934196
:102514008908591889004018e5e770bdd8000020e3
:0825240000000020c00a0000c5
:020000040000fa
:10252c0070b50e001c4c022310220100200000f09c
:10253c0075f81a4d23782b7063786b703178022301
:10254c001022200000f06af82378ab706378eb70ef
:10255c00717802231022200000f060f823782b7190
:10256c0063786b71b17802231022200000f056f8ca
:10257c002378ab716378eb71f17802231022200081
:10258c0000f04cf823782b7263786b720023ab72db
:10259c00280000f033fa70bd30040020b80300208e
:020000040000fa
:1025ac00f0b585b001900e00140001f08ff90128f0
:1025bc001ad1731efe2b17d8050002ab1e71002713
:1025cc00af4220d003abd95da368013ba360002bc5
:1025dc0004daa269934219db0a2917d023685a1c22
:1025ec00226019700137ebe723003200583303a93e
:1025fc00019800f079fc0500431ce0d14023060053
:10260c00a2891343a381300005b0f0bd22000198cc
:0c261c00fff7f0fd431ce5d10600f4e7d9
:020000040000fa
:10262800f0b583b0019300251a4b6c1ce4b2b1fbe2
:10263800f2f617007743c91b595531002500002ec3
:10264800f3d1019bfcb121000126124a94463027a0
:102658000fe0821865466d18013d2d78092d0fd9b8
:102668003735edb215700139c9b2721cd2b259b101
:102678001600721ed2b29c42ebda8754013bf4e793
:102688003035edb2eee7260000238355300003b065
:08269800f0bdc04698030020cc
:020000040000fa
:1026a00070b5184d184c2900200001f02ff82100ba
:1026b00010310422280001f039f878b90422134bb4
:1026c000da61134b1b78c3b10022114b1a70104b07
:1026d0001978c9b20c48183001f018f80d4b1b7866
:1026e00013b100220b4b1a70064b19004031002227
:1026f0001a7001338b42fbd170bd0122044b1a705a
:10270000e5e7c046a40200202c0100000032004092
:0827100017040020350400202d
:020000040000fa
:10271800f8b51c4b07001e68b36913b9300000f008
:10272800ddf84836b4687368013b03d5336833b1c4
:102738003668f7e70c22a55e6db16434f4e704212e
:10274800380000f099fe30600028f1d10c23040015
:102758003b602000f8bd01235b42e3812000012398
:102768002566a3812560a560656025616561a56111
:1027780008222900583001f08bf96563a563a56428
:08278800e564e6e7683b000090
:020000040000fa
:10279000f7b502268b8905000c00334206d02300d2
:1027a00047332360236101236361f7bd01ab6a46b0
:1027b00000f05afa009907002800fff781fd30b9b0
:1027c0000c22a35e9a05f0d41e43a681e7e70d4bc9
:1027d000ab628023a28920601343a381009b206108
:1027e0006361019b4bb10e23e15e280000f0feff08
:1027f00018b10123a2891343a381a0893843a08182
:08280000d3e7c046a93a00002d
:020000040000fa
:1028080053756e64617900004d6f6e6461790000e4
:1028180054756573646179005765646e65736461a6
:1028280079000000546875727364617900000000d3
:1028380046726964617900005361747572646179e4
:10284800000000004a616e00466562004d6172003a
:10285800417072004d6179004a756e004a756c00ce
:1028680041756700536570004f6374004e6f7600c2
:042878004465630050
:020000040000fa
:10287c00174a137801210b431370110001224b6886
:10288c001a42fcd1124a1378102110200343137002
:10289c00a023d3610223936113610e4b19720120a3
:1028ac001875202019542c20195438201954442000
:1028bc001954502019545c201954137802210b43dd
:1028cc001370110002224b681a42fcd17047c046ab
:0828dc00002a0040000000206a
:020000040000fa
:1028e400836913b5040043bb8364c3640365134b5a
:1028f400134a1b6882620193984201d101238361c8
:102904002000fff707ff60602000fff703ffa060cf
:102914002000fff7fffe0022e0600421606800f061
:102924005bfa01220921a06800f056fa0222122162
:10293400e06800f051fa0123a36113bd683b000075
:04294400a93a0000ac
:020000040000fa
:102948000122144b1a601a00d369002bfcd140f203
:102958000012104b5a601a00d369002bfcd10d4ba2
:102968000122da600c4a1a601a00d369002bfcd1e4
:102978001022084b5a831a00d369002bfcd1074b4d
:10298800002221215a5420215a548322014b9a753e
:102998007047c0460004004216002000440300208f
:020000040000fa
:1029a800f0b530b3144b1a7d002302bb124b1860ec
:1029b800596001221a750023104c0126072702e0ee
:1029c800c25c228501331d00227e324209d0994221
:1029d80007d062683a40012af2d15a00825a228509
:1029e800f0e7054b9d600122044b9a7501231800fe
:1029f800f0bd0023fbe7c046140300200008004296
:020000040000fa
:102a080010b588b004006a46134b4c3303cb03c29d
:102a18001b881380162200210a20684401f038f828
:102a280000231a006a44e15c517201330a2bf8d181
:102a38000d236a46d3740023137513216846fff7e4
:102a4800afff01f051f80028fbd1694602486c300d
:0c2a580000f058fe08b010bd2c0100007a
:020000040000fa
:102a640070b504000d0010b300f0c6fccdb1200019
:102a74000024104a0421072605e0138d0380023048
:102a84000134a5420ed0137e0b42fcd0538b33424b
:102a940008d153683340012befd0138d03700130fc
:102aa400eee700242c1b60426041c0b270bd0020e0
:082ab400fce7c046000c0042e3
:020000040000fa
:102abc00114b124a1a60124a9a81c02292025a6031
:102acc001a00d369002bfcd10b4a136802210b436b
:102adc001360d369002bfcd10a4b00229a61da6196
:102aec001a622c215a545a621a605a609a601a75ea
:102afc00da60da857047c0460008004204011041d4
:082b0c005bb1ffff1403002080
:020000040000fa
:102b140070b586b001ac0025019502950395049526
:102b24002582a57421700133012b0bdd01250121c0
:102b340026005418013c247874550131c9b20d00a3
:102b44009942f6db00881a0001a900f06bfb05002e
:102b540000f03cfd04000028fad100f083ff00b12e
:082b64002500280006b070bd39
:020000040000fa
:102b6c00c3685b0482681203134302681343426810
:102b7c00920113434269743a92061343026901327b
:102b8c00920513430a4a13621000202203691a4269
:102b9c00fcd12423064ad154110040f600020b69e3
:102bac001a42fcd140f20012014b5a8101207047ad
:042bbc0000240040b1
:020000040000fa
:102bc00010b5114b00229a61da61104b83221a76fc
:102bd0005a680f4c22405a601a00d369002bfcd16e
:102be00061b103242023084ad45440000843074b12
:102bf00058621a00d369002bfcd110bd0424202395
:102c0000014ad454f1e7c0464403002000040042c6
:042c1000fffffbffc8
:020000040000fa
:102c14000b6970b505000c000bb9002070bd18b12c
:102c240083690bb9fff75cfe0b4b9c4209d16c68be
:102c34000c22a35e002bf0d021002800fef70eff2b
:102c4400ece7064b9c4201d1ac68f1e7044b9c4293
:102c5400eed1ec68ece7c0466c3700008c3700001e
:042c64004c370000e9
:020000040000fa
:102c680070b50e001d000e23c95e90b01400002937
:102c780007da00232b60b3891b0611d440f2004306
:102c88000fe001aa00f0d6fc0028f2db4ff20002a8
:102c9800029b1340054a9b185a4253412b60ede7ab
:102ca80040230020236010b070bdc04600e0ffff45
:020000040000fa
:102cb80010b5002402238b4264410419e4b20cb11c
:102cc800013a92b24b005b18db00591a092091fbbc
:102cd800f0f000190430910840186423b2fbf3f3b4
:102ce800c01a40f29013b2fbf3f28218072092fb4d
:0c2cf800f0f0c300181a101ac0b210bd92
:020000040000fa
:102d0400104b04221a60022243215a5444215a547b
:102d1400012248215a5449215a544a215a545021d3
:102d24005a5451215a5456215a5457215a54332132
:102d340034229954222238215a543b215a540022d5
:082d4400da667047003200401e
:020000040000fa
:102d4c0010b50a4b98470a4b9847fff7a5fb094a61
:102d5c007f21094b8b439360084b9847084b98474e
:102d6c00084b984700f002fafee7c0462f350000ea
:102d7c002f35000000ed00e000000000952d000054
:082d8c002f3500002f35000077
:020000040000fa
:102d940070b500260c4d0d4c641ba410a64209d13d
:102da4000026fdf7adf90a4d0a4c641ba410a64297
:102db40005d170bdb300eb5898470136eee7b30078
:102dc400eb5898470136f2e71001000010010000ab
:082dd4001001000014010000d1
:020000040000fa
:102ddc00002310b5040003604360836081810366a7
:102dec00c28103614361836119000822583000f0ed
:102dfc004dfe054b24626362044ba362044be362f9
:102e0c00044b236310bdc046a9350000613200009d
:082e1c00ad340000093b000089
:020000040000fa
:102e2400f8b50d00096e06001400d718890418d5ea
:102e34009f08bf00d719bc4201d1002008e02a0036
:102e440002cc300000f0f0fc431cf4d101204042dd
:102e5400f8bd21782a00300000f052fb0134431cf5
:082e6400f4d0bc42f5d1e8e70f
:020000040000fa
:102e6c0010b504220e4b5a6000f07afafff744ffbb
:102e7c00fef7feff00f0eafd00f024fafff718fe63
:102e8c00fef73dfbfff75afd00f0aefbfff7f0fc41
:102e9c0000f0eef800f07cfafef76cff10bdc046b7
:042eac000050004191
:020000040000fa
:102eb00001220d4b1a700d4b1b78dbb22bb1012b8d
:102ec0000ad00022094b1a7005e00422084b9a61cf
:102ed0000122064b1a7070470422054b5a610022ea
:102ee000024b1a70f7e7c0461604002017040020b2
:042ef000003200406c
:020000040000fa
:102ef4007fb51d000d4b04001b681b6a81b903b923
:102f04000b4be0331e6800222b0001a92000b047c0
:102f1400431c03d100232b608a23236004b070bdbb
:102f240003b9034be0331e682b00efe720040020b5
:042f3400d8000020a1
:020000040000fa
:102f3800f7b5050c019393b21f006b439c46140c24
:102f480086b277436643654366443c0ca419a342a2
:102f580002d980235b02ed18260cbfb2019b240422
:102f6800e41943432000514375195918491903b00e
:022f7800f0bdaa
:020000040000fa
:022f7a00fee770
:020000040000fa
:102f7c0010b5054c237833b9044b13b1044800e069
:102f8c0000bf0123237010bdd803002000000000f7
:102f9c0000000000034b10b51bb10349034800e0cf
:102fac0000bf10bd00000000dc030020000000008a
:020000040000fa
:102fbc0010b50e4948f200020b691a42fcd10b4bba
:102fcc009b691a0b1f210a4082609c093f22144006
:102fdc0044601a4002609a01120f013a02619a0e83
:102fec00743242615b0c0b40c36010bd0024004086
:020000040000fa
:102ffc0030b5b0b1b9b10d4a0124072503e00388ff
:10300c001385023059b10139137e2342fcd0536829
:10301c002b40012bf3d0037813850130f2e701200c
:10302c0030bd0020fce70120fae7c046000c00424e
:020000040000fa
:10303c0070b504000d00a0b12c230b4ad35c00200a
:10304c0003b170bd00f0eaf9074b9c61dd61002211
:10305c001a6201202c215854da858422034b9a756c
:10306c00efe70020ede7c046140300200008004203
:020000040000fa
:10307c0001220d4b1a6019000b691a42fcd10a4b44
:10308c0040f218721a6003221a7340f2d032da61dd
:10309c0033229a720021054a116001225a721a00d9
:1030ac001369002bfcd1704700100042180400205b
:020000040000fa
:1030bc00002b11d1002a0fd1002900d1002802d0f9
:1030cc000021c943081c07b4024802a14018029011
:1030dc0003bdc046850a000003b4684601b50298da
:1030ec00fef778f8019b9e4602b00cbc7047c046b8
:020000040000fa
:1030fc00f7b5040007000026019148340cb93000e4
:10310c00febd6368a5680093009b013b009301d54d
:10311c002468f3e7ab89012b08d90e22ab5e01338f
:10312c0004d029003800019b984706436435ebe72f
:020000040000fa
:10313c00c3685b048268120313430268134342683a
:10314c00920113434269743a9206134302690132a5
:10315c0092051343044a9361110008220b691a4229
:0c316c00fcd101207047c0460024004048
:020000040000fa
:1031780010b582b048f200031c680020fff772fe09
:10318800631c0ed084f3888848f204031b680193fb
:10319800019c64086400200021002200230000f044
:0c31a800c7f8fdf769fe012002b010bd61
:020000040000fa
:1031b4001c2101231b04984201d3000c10391b0a63
:1031c400984201d3000a08391b09984201d3000927
:1031d400043902a2105c40187047c046040302027e
:0c31e400010101010000000000000000db
:020000040000fa
:1031f00070b5050020230b4ce35c002003b170bdcb
:10320000a580e16062610022a26022610121a170bb
:1032100022702121625401212800fff7d1fc0120f6
:08322000ede7c0464403002065
:020000040000fa
:1032280070b5050020230b48c35c002003b170bdb6
:10323800084b9d800024dc605c6199601a619c7079
:103248001c7021229c5400212800fff7b5fc0120a6
:08325800ede7c046440300202d
:020000040000fa
:10326000f8b51f008b8905000c001600db0505d59d
:103270000e23c95e0022022300f0f2f9a389054a59
:1032800028001340a38132000e23e15e3b0000f0d2
:08329000c3f9f8bdffefffffd9
:020000040000fa
:1032980070b50c00002519b112b11500022801d92a
:1032a800280070bd074b23b11100200000e000bfcb
:1032b800f6e716002078013e00f025fb0134002ec9
:0832c800f8d1ede70000000061
:020000040000fa
:1032d0000a4b0b4a1a6041f212429a81c0229202b2
:1032e0005a601a00d369002bfcd1044a13680221ea
:1032f0000b431360d369002bfcd17047000c0042d4
:043300000441104133
:020000040000fa
:103304003031323334353637383941424344454617
:1033140000303132333435363738396162636465ad
:103324006600232d302b2000686c4c0065666745d1
:0333340046470009
:020000040000fa
:10333800e0b545464e465746e0b45d4620b42546be
:1033480026462746a046a146a246a346a44684f39d
:103358000088a44720bcab46e0bcba46b146a846a4
:02336800e0bdc6
:020000040000fa
:02336a00fee77c
:020000040000fa
:10336c000a4b00221a819a7901210a439a719b789f
:10337c0003221340022b07d00222044b9a7019002f
:10338c0001228b791342fcd07047c04600040040e8
:020000040000fa
:10339c00094a138801210b431380110001220b6988
:1033ac001a42fcd1054a044b1a80190002220b69ff
:1033bc001a42fcd17047c046002400400a8bffff24
:020000040000fa
:1033cc00094b1b68db439b0700d07047074b996880
:1033dc0040f2e8335843b0fbf3f0044a93685b1aad
:1033ec009842fbd8f1e7c04610e000e060000020f6
:020000040000fa
:1033fc00094b5b8b5b070dd0074b80221a7607229b
:10340c005a831b7e5b0705d5034b04211a8d1a7e4c
:0c341c000a42fbd17047c046000c004281
:020000040000fa
:10342800094b5b8b5b070dd0074b80221a7607226e
:103438005a831b7e5b0705d5034b04211a8d1a7e20
:0c3448000a42fbd17047c0460008004259
:020000040000fa
:1034540010b5084b5b7a5bb1064b987ac0b2332245
:103464009a7228b1044b1b6813b1034a51689847f8
:0c34740010bdc0460010004218040020eb
:020000040000fa
:1034800070b564254a1e55430e0029007031fef7c1
:1034900017ff040040b100212a00016046600c3093
:0c34a000a060643200f0f8fa200070bd5b
:020000040000fa
:1034ac0070b50c000e25495f00f0d4f8a389421cbe
:1034bc0003d1054a1340a38170bd41f200021343ae
:0c34cc00a3816065f8e7c046ffefffff3a
:020000040000fa
:1034d800074a13684bb107491818884202d8106088
:1034e8001800704701204042fbe7034b1360f2e7e6
:0c34f8002c0400204006002040040020ae
:020000040000fa
:10350400936810b5013b9360002b05da9469a342dc
:1035140008dbcbb20a2b05d01368581c1060197055
:0a352400c8b210bdfef76afefbe717
:020000040000fa
:02352e007047e4
:020000040000fa
:1035300030b543001b189b00064ce3181b7a8342ee
:1035400000d030bd43001d18ad0029516019426004
:08355000f7e7c046000000206f
:020000040000fa
:1035580010b5064a908980b2054b186005499181db
:103568005b6813b1024a9168984710bd0024004077
:0835780000040020ffc1ffff69
:020000040000fa
:1035800010b5064a1378591c117005480178054a90
:10359000d1540121fff752fd10bdc0463504002073
:0835a00036040020a402002003
:020000040000fa
:1035a80070b50c000e25495f00f068f8002803dbb1
:1035b800636d1b18636570bda389024a1340a3811c
:0835c800f9e7c046ffefffff29
:020000040000fa
:1035d0002023064ad35c01203bb9054b588b30238e
:1035e00018401038431e9841c0b270474403002071
:0435f0000004004291
:020000040000fa
:1035f400064a00231360936040f2e73151600621cc
:103604001160034a936013607047c04610e000e005
:043614006000002032
:020000040000fa
:1036180070b50500080011000022054c22601a0050
:1036280000f094fa431c02d1236803b12b6070bdeb
:04363800d40000209a
:020000040000fa
:10363c00002370b5064c050008001100236000f053
:10364c0073fa431c02d1236803b12b6070bdc046d2
:04365c00d400002076
:020000040000fa
:1036600070b50500080011000022054c22601a0008
:1036700000f068fa431c02d1236803b12b6070bdcf
:04368000d400002052
:020000040000fa
:1036840070b50500080011000022054c22601a00e4
:1036940000f05afa431c02d1236803b12b6070bdb9
:0436a400d40000202e
:020000040000fa
:1036a80070b5002661b15ab1160048b90c00150072
:1036b800012000f01bf9013d20700134002df7d1e5
:0436c800300070bda1
:020000040000fa
:1036cc0010b50222044b5a61044bdb6813b1034a58
:1036dc001069984710bdc046002a00400000002029
:020000040000fa
:1036ec0070b50088fff77efd0500fff76bff040047
:1036fc000028fad100f0b2f900b12500280070bd05
:020000040000fa
:10370c000fb407b5054b04aa1b6802ca986801924e
:10371c0000f05af903b008bc04b01847200400208c
:020000040000fa
:10372c0030b5002352b1013ac45ccd5cac4204d13b
:10373c009a4202d00133002cf6d1631b180030bd25
:020000040000fa
:10374c00000000000000000000000000000000006d
:10375c00000000000000000000000000000000005d
:020000040000fa
:10376c00000000000000000000000000000000004d
:10377c00000000000000000000000000000000003d
:020000040000fa
:10378c00000000000000000000000000000000002d
:10379c00000000000000000000000000000000001d
:020000040000fa
:1037ac00002370b5054c050008002360fff78efe62
:1037bc00431c02d1236803b12b6070bdd4000020e0
:020000040000fa
:1037cc00002370b5054c05000800236000f0a8f933
:1037dc00431c02d1236803b12b6070bdd4000020c0
:020000040000fa
:1037ec00002370b5054c05000800236000f0a0f91b
:1037fc00431c02d1236803b12b6070bdd4000020a0
:020000040000fa
:10380c0082b001b901a910002ab133b113780b6051
:10381c001078431e984102b0704702204042fae7ec
:020000040000fa
:10382c0010b50c23d45e42f200031c4204d11c439d
:0e383c009481146e23431366fef7b2fe10bd96
:020000040000fa
:02384a007047c5
:020000040000fa
:10384c00044a536804490b405360d369002bfcd1e4
:0c385c007047c046000c0042fffffeff5a
:020000040000fa
:10386800044a536804490b405360d369002bfcd1c8
:0c3878007047c046000c0042fffffdff3f
:020000040000fa
:10388400044a536804490b405360d369002bfcd1ac
:0c3894007047c04600080042fffffeff26
:020000040000fa
:1038a000044a536804490b405360d369002bfcd190
:0c38b0007047c04600080042fffffdff0b
:020000040000fa
:1038bc0010b5054b9a6801329a601b6813b1024a25
:0c38cc005068984710bdc0466000002006
:020000040000fa
:1038d800044b1b681b6a03b9034b40f22812985c1f
:0c38e8007047c04620040020d8000020db
:020000040000fa
:1038f40000b583b000230193012101a8fff7b0f8bc
:0a3904000028f9d0019803b000bdbf
:020000040000fa
:10390e0000b583b06b46d87101216b46d81dfff709
:0a391e006efb0028f8d003b000bdd6
:020000040000fa
:1039280083788b6043784b6003780b60c378cb60f7
:0a39380003790b61c3884b617047ef
:020000040000fa
:023942007047cc
:020000040000fa
:103944000422044b5a7019004b781342fcd030bf48
:083954007047c046000400406a
:020000040000fa
:10395c00044a516880235b020b435360d369002bec
:08396c00fcd17047000c004281
:020000040000fa
:10397400044a516880239b020b435360d369002b94
:08398400fcd17047000c004269
:020000040000fa
:10398c00044a516880235b020b435360d369002bbc
:08399c00fcd170470008004255
:020000040000fa
:1039a400044a516880239b020b435360d369002b64
:0839b400fcd17047000800423d
:020000040000fa
:1039bc00c20f0000221000003c1000001e1100007d
:0839cc003c110000481100004d
:020000040000fa
:1039d40010b513000a00010002480068fcf778fee5
:0839e40010bdc04620040020c4
:020000040000fa
:1039ec000b0021b1ff2a04d98a2303608b3b1800fa
:0839fc0070470a700123fae78d
:020000040000fa
:103a0400c9b28218904201d10020704703788b42da
:063a1400fbd00130f6e7d3
:020000040000fa
:103a1c00034b00229a601a6801210a431a6070470e
:043a2c0010e000e0c6
:020000040000fa
:103a300010b50400fff7f2ff2000fff7c7fc00f00d
:043a40001bf810bda2
:020000040000fa
:103a440010b5034b01001868fef76efb10bdc046ad
:043a5400200400202a
:020000040000fa
:103a5800024b00225a6001221a727047005000413e
:020000040000fa
:103a68002123024ad05cc0b27047c04644030020fc
:020000040000fa
:103a7800024a136801218b431360704710e000e08d
:020000040000fa
:103a8800c30502d50122014b1a70704715040020a6
:020000040000fa
:103a980003008218934200d1704719700133f9e787
:020000040000fa
:103aa80010b50249fff726fb10bdc046152c0000d3
:020000040000fa
:0e3ab80010b54a1c097884680123a04710bd90
:020000040000fa
:0e3ac6000180c2608360009b43600120704756
:020000040000fa
:0e3ad4000023c25c0133002afbd1581e70474c
:020000040000fa
:0c3ae400014b58609960704700040020fe
:020000040000fa
:0c3af000014b187dc0b270471403002089
:020000040000fa
:0c3afc00014b58629962704714030020cf
:020000040000fa
:0c3b080010b50e23c95efff75dfe10bd76
:020000040000fa
:0c3b140042f2000300204b607047c046e6
:020000040000fa
:0b3b20004300504f53495800002e0096
:020000040000fa
:083b2c0010b500f015f810bd02
:020000040000fa
:083b340010b5fff7edff10bd15
:020000040000fa
:083b3c0010b500f015f810bdf2
:020000040000fa
:083b440010b500f013f810bdec
:020000040000fa
:083b4c0010b5fff7abfd10bd41
:020000040000fa
:083b540010b5fff79ffb10bd47
:020000040000fa
:083b5c00012040427047c04601
:020000040000fa
:043b64007047c046a0
:020000040000fa
:043b680044020020f3
:020000040000fa
:043b6c00012070477d
:020000040000fa
:043b7000002070477a
:020000040000fa
:087e00007fe97fe9f8f776b98c
:020000040000fa
:0200000400807a
:044000007f438fb0bb
:020000040000fa
:0200000400807a
:04400400bbfcffff03
:020000040000fa
:0200000400807a
:0440080080d0f8c0ac
:020000040000fa
:0200000400807a
:04400c00ffffffffb4
:020000040000fa
:0200000400807a
:0440100000000000ac
:020000040000fa
:0200000400807a
:0440140002000000a6
:020000040000fa
:0200000400807a
:0440180000000000a4
:020000040000fa
:0200000400807a
:04401c001e65338466
:020000040000fa
:0200000400807a
:04c00000ff00c0a0dd
:020000040000fa
:0200000400807a
:04c0040000ffffff3b
:020000040000fa
:0200000400807a
:04c008004081e7ddaf
:020000040000fa
:0200000400807a
:04c01000ffffffff30
:020000040000fa
:0200000400807a
:04c01400ffffffff2c
:020000040000fa
:0200000400807a
:04c01800ffffffff28
:020000040000fa
:0200000400807a
:04c01c00ffffffff24
:020000040000fa
:0200000400807a
:04c02000ffffffff20
:020000040000fa
:0200000400807a
:04c02400ffffffff1c
:020000040000fa
:0200000400807a
:04c02800ffffffff18
:020000040000fa
:0200000400807a
:04c02c00ffffffff14
:020000040000fa
:0200000400807a
:04c03000ffffffff10
:020000040000fa
:0200000400807a
:04c03400ffffffff0c
:020000040000fa
:0200000400807a
:04c03800ffffffff08
:020000040000fa
:0200000400807a
:04c03c00ffffffff04
:020000040000fa
:0200000400807a
:04c04000ffffffff00
:020000040000fa
:0200000400807a
:04c04400fffffffffc
:020000040000fa
:0200000400807a
:04c04800fffffffff8
:020000040000fa
:0200000400807a
:04c04c00fffffffff4
:020000040000fa
:0200000400807a
:04c05000fffffffff0
:020000040000fa
:0200000400807a
:04c05400ffffffffec
:020000040000fa
:0200000400807a
:04c05800ffffffffe8
:020000040000fa
:0200000400807a
:04c05c00ffffffffe4
:020000040000fa
:0200000400807a
:04c06000ffffffffe0
:020000040000fa
:0200000400807a
:04c06400ffffffffdc
:020000040000fa
:0200000400807a
:04c06800ffffffffd8
:020000040000fa
:0200000400807a
:04c06c00ffffffffd4
:020000040000fa
:0200000400807a
:04c0e000ffffffff60
:020000040000fa
:0200000400807a
:04c0e400ffffffff5c
:020000040000fa
:0200000400807a
:04c0e800ffffffff58
:020000040000fa
:0200000400807a
:04c0ec00ffffffff54
:020000040000fa
:0200000400807a
:04c0f000ffffffff50
:020000040000fa
:0200000400807a
:04c0f400ffffffff4c
:020000040000fa
:0200000400807a
:04c0f800ffffffff48
:020000040000fa
:0200000400807a
:04c0fc00ffffffff44
:00000001FF
